:020000040000FA
:06000000E6EF1DF0120006
:0600080004EF10F01200ED
:060018000CEF10F01200D5
:06200000E6EF1DF01200E6
:06200800B7EF18F0120012
:06201800C0EF18F01200F9
:06202A0001000E3C000065
:08203000600000004E000000FA
:08203800D9CFE6FFE1CFD9FF8B
:10204000E652A09A6A6A686A160E6F6E9F0E6B6EF1
:102050007B0E696E6D8C6E6A010EE66EE66AE66A4C
:10206000710EE66E0F0EE66EBCEC1DF00B6E050EEB
:10207000E15E0B506D9CDF6ADF500B6E0C6A080E40
:102080000B5C000E0C5810E2DF50040DF3CFE9FF9B
:10209000F4CFEAFF000EE926040EEA22EE6AEE6AA9
:1020A000EE6AEE6ADF2AE8D7160E706E68A602D0D6
:1020B0006896FCD70001C16BC66BC76BC86B6D9887
:1020C000DF6A020EDF5C18E2EA6ADF34FE0BEA36F2
:1020D000E96EB90EE926000EEA22EE6AED6AEA6AB6
:1020E000DF34FE0BEA36E96EB50EE926000EEA2271
:1020F000EE6AED6ADF2AE5D70001080EB96F040E1B
:10210000BA6FAF6BAE6BE552E552E7CFD9FF120065
:10211000D9CFE6FFE1CFD9FFE6520001AE5116E17B
:1021200006D06D6A696A0001AE6BA19AA8D06D6A8B
:10213000696A160E6F6E9F0E6B6E7B0E696E6DB6C2
:1021400002D06D86FCD70001010EAE6FAE0508E12E
:102150006DBA06D0686A696A69806988020EAE6FD6
:102160006850040B05E06950040B02E06894B7D88E
:102170006DA202D0A19A83D06850010B12E0695081
:10218000010B0FE059DF0001040EAE6F0401200EB9
:10219000026F040E036F080E016F006B8C0E0013AC
:1021A00068906850100B05E06950100B02E085D86C
:1021B00068986850400B13E06950400B10E0010E26
:1021C000E66EE66A000EE66EE66A730EE66EE66A94
:1021D0003FEC1CF00B6E060EE15E0B50689C6850E5
:1021E000200B04E06950200B01E04ED86850020B30
:1021F00013E06950020B10E0010EE66EE66A000E75
:10220000E66EE66AE6687F0EE66E3FEC1CF00B6E4B
:10221000060EE15E0B506A6A040E0001E76EAE190D
:10222000E8AE02D0E73402D0E750AE5D02E2A19AF8
:1022300026D069A623D0DF6A040EDF5C1FE268A601
:102240001AD06CCFCEF06896780E0001CE1502E160
:102250005BD810D0000EE66EE66ACE0EE66E000E7B
:10226000E66E720EE66EE66A3FEC1CF00B6E060E32
:10227000E15E0B5001D002D0DF2ADED7A19AE552F1
:10228000E552E7CFD9FF120070A015D0B1C0E9FF29
:10229000B2C0EAFFEF5080080DE1B9C0E9FFBAC053
:1022A000EAFFEF50840806E1B1C0E9FFB2C0EAFFDF
:1022B0008C0EEF6E7090689A1200698468986D8237
:1022C000000EE66EE66AE66EE66A750EE66EE66A91
:1022D0003FEC1CF00B6E060EE15E0B501200000E80
:1022E000E66EE66AE66EE66A740EE66EE66A3FEC55
:1022F0001CF00B6E060EE15E0B506D92699468A4A3
:1023000002D06894FCD71200D9CFE6FFE1CFD9FF05
:10231000E652FD0E0001CE155AE17E0ECE15E840C4
:102320007F0B040DF3CFB1F0F4CFB2F0000EB12764
:10233000040EB223B1C0B3F0B2C0B4F0B375B1C0F3
:10234000E9FFB2C0EAFFEF503C0BE842E8420D085B
:102350003CE1B1C0E9FFB2C0EAFF020EE926000E7F
:10236000EA22EECF0BF0EFCF0CF0280E0B1802E1B3
:10237000040E0C1828E1B1C0E9FFB2C0EAFF020E5A
:10238000E926000EEA22200EEE6E040EED6EDF6AE4
:10239000DF500B6E0C6A080E0B5C000E0C5813E23B
:1023A000DF50EA6A280FE96E040EEA22EF50E66E6B
:1023B000DF50EA6A200FE96E040EEA22E552E75088
:1023C000EF6EDF2AE5D70DD801D02ED805D0FD0E4F
:1023D000CE15040801E14ED8E552E552E7CFD9FF0A
:1023E0001200B9C0E9FFBAC0EAFFEF50800B05E068
:1023F000B9C0E9FFBAC0EAFFEF6A0001BD6BBE6B6E
:10240000C26BC36BC16BB6D8000EE66EE66AE66EB1
:10241000E66A030EE66EE66A3FEC1CF00B6E060EF3
:10242000E15E0B5065EF14F0020E0001BE5D02E1AB
:10243000ACDB1FD06CD80001CF511AE1B3C0E9FF6B
:10244000B4C0EAFFEE52080EEF6EB3C0E9FFB4C0AD
:10245000EAFF020EE926000EEA22200EEE6E040EBE
:10246000ED6EB3C0E9FFB4C0EAFF8C0EEF6E01D091
:10247000CF6B1200D9CFE6FFE1CFD9FFE652B9C04A
:10248000E9FFBAC0EAFFEF50400B01E0010EDF6E3A
:102490000001B975080EAE5D0AE122C46EFF6E50F0
:1024A000000803E2100EAE6F02D0040EAE6FBE0540
:1024B00028E1B9C0E9FFBAC0EAFF020EE926000E22
:1024C000EA22280EEE6E040EED6ED4DA020E000142
:1024D000BD5D07E1B9C0E9FFBAC0EAFF840EEF6E47
:1024E0000FD0DF5007E1B9C0E9FFBAC0EAFFC80E5C
:1024F000EF6E06D0B9C0E9FFBAC0EAFF880EEF6EF2
:1025000001D005D8E552E552E7CFD9FF1200D9CF67
:10251000E6FFE1CFD9FF020EE1260001BE6BB9C094
:10252000E9FFBAC0EAFFEF6A040EB9190B6EBAC030
:102530000CF00BC0DEFF0CC0DDFFDECFE9FFDDCF0E
:10254000EAFFEF6AC6AF0CD0C951CA1107E005D047
:10255000CAC0FAFF0001C951F96EFADF0001C69F37
:10256000020EE15C02E2E16AE552E16EE552E7CF7C
:10257000D9FF120004012051600BE842E842E84212
:10258000E842E842000901E058D021510C0A54E029
:102590000B0A43E00C0A35E0010A26E00B0A22E0B0
:1025A000020A20E0030A1CE0080A10E0010A0CE01D
:1025B0000F0A08E0030A01E03FD00001C18F080EB6
:1025C000AE6F3BD0C7D839D07DDB37D00001AF0E1E
:1025D000BF6F000EC06FC181010EC26FC18F2DD0C1
:1025E00013D92BD02BD829D024510001BF6FC06B39
:1025F000B00EBF27000EC023C181010EC26FC18F74
:102600001CD00001C18F04012451EA6AB00FE96EA9
:10261000000EEA2222C4EFFF10D0000EE66EE66A3A
:10262000E66EE66A020EE66EE66A3FEC1CF00B6EA2
:10263000060EE15E0B5001D000D01200D9CFE6FFAC
:10264000E1CFD9FF040EE1260401220510E120515B
:102650001F0B00090CE10001C18F030E0401215D75
:1026600004E10001010ECD6F02D00001CD6B040129
:10267000225166E120511F0B020862E124510F0B29
:1026800000095EE00001C18F040124BF10D0245175
:102690000F0BE96EEA6AD890E936EA36B50EE926FC
:1026A000000EEA22EECFDEFFEDCFDDFF0FD024518A
:1026B0000F0BE96EEA6AD890E936EA36B90EE926D8
:1026C000000EEA22EECFDEFFEDCFDDFF030E215D2F
:1026D00007E1DECFE9FFDDCFEAFF840EEF6E30D0F9
:1026E00024510F0B0C6A700F0B6E0F0E0C22020E92
:1026F0000BC0DBFF030E0CC0DBFF020EDBCFE9FFDC
:10270000030EDBCFEAFFEF9024AF0DD0DECFE9FF61
:10271000DDCFEAFFEF6ADF74DECFE9FFDDCFEAFF4E
:10272000400EEF6E0DD0DECFE9FFDDCFEAFF880E61
:10273000EF6EDF74DECFE9FFDDCFEAFFC80EEF6E8C
:10274000040EE15C02E2E16AE552E16EE552E7CF98
:10275000D9FF1200800E0401205D55E10001C00E7A
:10276000C16F04012351030A2EE0010A0EE0030A9F
:1027700003E00001C16B47D00001140EBF6F390E9A
:10278000C06F120EC26FC36B3ED02251F66EF76A55
:10279000D890F636F736F40EF626390EF7220900F1
:1027A000F5CFBFF00A00F5CFC0F0020E0001F76AC6
:1027B000BF25F66EC051F7220900F5CFC2F00A001E
:1027C000F5CFC3F020D0030E225D1AE22251F66E3F
:1027D000F76AD890F636F736F60EF626390EF72257
:1027E0000900F5CFBFF00A00F5CFC0F0BFC0F6FF7B
:1027F000C0C0F7FF0800F5500001C26FC36B02D0E4
:102800000001C16B00D01200D9CFE6FFE1CFD9FFA4
:10281000020EE1260401286B296B20511F0B020ACE
:1028200012E0030A0DE0010A01E03BD00001C18F74
:10283000040128810001CD0502E10401288331D083
:102840000001C18F2ED00001C18F040124BF10D020
:1028500024510F0BE96EEA6AD890E936EA36B50ED4
:10286000E926000EEA22EECFDEFFEDCFDDFF0FD02E
:1028700024510F0BE96EEA6AD890E936EA36B90EB0
:10288000E926000EEA22EECFDEFFEDCFDDFFDECF40
:10289000E9FFDDCFEAFFEF50040B02E0010E286FE5
:1028A00000D00001C1AF07D0280EBF6F040EC06F6B
:1028B000C181020EC26F020EE15C02E2E16AE552E2
:1028C000E16EE552E7CFD9FF12006D980001C1BF5C
:1028D0004AD0C6AF28D0020EBE6FB9C0E9FFBAC059
:1028E000EAFFEE52EF6AB9C0E9FFBAC0EAFFC80ECC
:1028F000EF6EB3C0E9FFB4C0EAFFEE52080EEF6E10
:10290000B3C0E9FFB4C0EAFF020EE926000EEA22D6
:10291000280EEE6E040EED6EB3C0E9FFB4C0EAFF00
:10292000C80EEF6E1FD0B3C0E9FFB4C0EAFFEE528D
:10293000080EEF6EB3C0E9FFB4C0EAFF020EE9264D
:10294000000EEA22200EEE6E040EED6EB3C0E9FF1B
:10295000B4C0EAFF8C0EEF6EB9C0E9FFBAC0EAFF5F
:10296000840EEF6E86D0C6BF84D0040120AF59D04C
:102970000001C2510401265D0001C3510401275921
:1029800004E226C4C2F027C4C3F074D80001010ECB
:10299000BE6FB3C0E9FFB4C0EAFFEE52080EEF6E9F
:1029A000B3C0E9FFB4C0EAFF020EE926000EEA2236
:1029B000200EEE6E040EED6EB3C0E9FFB4C0EAFF68
:1029C000800EEF6ECF6BB1C0E9FFB2C0EAFFEE52EE
:1029D000080EEF6EB1C0E9FFB2C0EAFF020EE926B1
:1029E000000EEA22200EEE6E040EED6EB1C0E9FF7D
:1029F000B2C0EAFF840EEF6E010ECF6FB9C0E9FFDF
:102A0000BAC0EAFF020EE926000EEA22280EEE6E98
:102A1000040EED6EB9C0E9FFBAC0EAFFC80EEF6E52
:102A200028D00001020EBE6FB9C0E9FFBAC0EAFFAC
:102A3000EE52EF6AB9C0E9FFBAC0EAFFC80EEF6E06
:102A4000B3C0E9FFB4C0EAFFEE52080EEF6EB3C0A8
:102A5000E9FFB4C0EAFF020EE926000EEA22280EC2
:102A6000EE6E040EED6EB3C0E9FFB4C0EAFFC80E0F
:102A7000EF6E1200D9CFE6FFE1CFD9FF020EE126BB
:102A80000001080EC25D000EC3590EE2C2C0DEFF97
:102A9000C3C0DDFFBD5103E1010EBD6F04D0BD0514
:102AA00002E1020EBD6F03D0080EDE6EDD6AB9C012
:102AB000E9FFBAC0EAFFEF92B9C0E9FFBAC0EAFF86
:102AC000EF90B9C0E9FFBAC0EAFF010EDB50EF1288
:102AD000B9C0E9FFBAC0EAFFEE52DFCFEFFF000E48
:102AE000DB50C25F010EDB50C35B280ECB6F040EC0
:102AF000CC6FC1B121D0D9CFE9FFDACFEAFFEE50D8
:102B0000ED1019E0BFC0F6FFC0C0F7FFBF2B000EED
:102B1000C0230800F550E66ECBC0E9FFCCC0EAFF49
:102B2000CB2B000ECC23E552E750EF6EDF06010EF3
:102B300001E2DB06E0D71FD0D9CFE9FFDACFEAFF09
:102B4000EE50ED1018E0BFC0E9FFC0C0EAFFBF2B98
:102B5000000EC023EF50E66ECBC0E9FFCCC0EAFF09
:102B6000CB2B000ECC23E552E750EF6EDF06010EB3
:102B700001E2DB06E1D7020EE15C02E2E16AE55226
:102B8000E16EE552E7CFD9FF1200D9CFE6FFE1CFE2
:102B9000D9FF020EE126B1C0E9FFB2C0EAFFEE5252
:102BA000EFCFDFFFDFCF0BF00B500001C75D000E52
:102BB000C85902E2C7C0DFFFDF500B6E0C6A0B5032
:102BC000C75DC76F0C50C859C86F010EDB6ADF5074
:102BD000F36E010EDBCFF4FFF350F45C16E2010E4E
:102BE000DB50EA6A280FE96E040EEA22EF50E66E27
:102BF000C4C0E9FFC5C0EAFFC42B000EC523E552DF
:102C0000E750EF6E010EDB2AE2D7000ED880C755E1
:102C1000000EC85528E2B3C0E9FFB4C0EAFFEE5287
:102C2000080EEF6EB3C0E9FFB4C0EAFF020EE9265A
:102C3000000EEA22280EEE6E040EED6EB1C0E9FF22
:102C4000B2C0EAFFEF50400B07E1B3C0E9FFB4C0E8
:102C5000EAFFC80EEF6E06D0B3C0E9FFB4C0EAFFCA
:102C6000880EEF6E25D0B3C0E9FFB4C0EAFFEE5284
:102C7000080EEF6EB3C0E9FFB4C0EAFF020EE9260A
:102C8000000EEA22200EEE6E040EED6EB3C0E9FFD8
:102C9000B4C0EAFF840EEF6EC951CA1107E005D037
:102CA000CAC0FAFF0001C951F96EFADF0001C69FE0
:102CB000020EE15C02E2E16AE552E16EE552E7CF25
:102CC000D9FF1200D9CFE6FFE1CFD9FFE6520001CC
:102CD000C18F010EE66EE66AE66A710EE66E0F0EB1
:102CE000E66EBCEC1DF00B6E050EE15E0B50DF6A6C
:102CF000DF500B6E0C6A080E0B5C000E0C5810E2D5
:102D0000DF50040DF3CFE9FFF4CFEAFF000EE92610
:102D1000040EEA22EE6AEE6AEE6AEE6ADF2AE8D76D
:102D20006D8C010EE66EE66AE66AB00EE66E000E87
:102D3000E66EBCEC1DF00B6E050EE15E0B506D9C5B
:102D40000001080EB96F040EBA6F000EB16F040EC9
:102D5000B26FB1C0B3F0B2C0B4F022C4AFF0AF51A3
:102D600003E1100EAE6F13D0010EE66EE66AAF0EF1
:102D7000E66E000EE66E010EE66EE66A3FEC1CF0B3
:102D80000B6E060EE15E0B500001200EAE6FE55299
:102D9000E552E7CFD9FF1200D9CFE6FFE1CFD9FF47
:102DA000020EE126000EDE6E040EDD6EFD0EDB501F
:102DB000E8240D6EFE0EDB50040DF3500D24040DBF
:102DC000F3500B6E0C6A020E0F0B05E0D8900C321C
:102DD0000B32E806FBE1D8900B360C36D8900B3658
:102DE0000C36D9CFE9FFDACFEAFF0B50EE260C50B4
:102DF000ED22DECFE9FFDDCFEAFFEF9EFD0EDB50D7
:102E00000FE1FE0EEA6ADB34FE0BEA36E96EB50E20
:102E1000E926000EEA22DECFEEFFDDCFEDFF0ED079
:102E2000FE0EEA6ADB34FE0BEA36E96EB90EE926DD
:102E3000000EEA22DECFEEFFDDCFEDFFDECFE9FFB1
:102E4000DDCFEAFFEF9CDECFE9FFDDCFEAFF040E26
:102E5000E926000EEA22EF8C020EE15C02E2E16A52
:102E6000E552E16EE552E7CFD9FF1200D9CFE6FF78
:102E7000E1CFD9FF020EE126FE0EDB500C6A700F87
:102E80000B6E0F0E0C220BC0DEFF0CC0DDFFDECF81
:102E9000E9FFDDCFEAFFFD0EDBCFEFFFDBA407D0BC
:102EA000E66AFE0EDBCFE6FF77DFE552E552FD0E68
:102EB000DBA208D0010EE66EFE0EDBCFE6FF6CDF74
:102EC000E552E552020EE15C02E2E16AE552E16E92
:102ED000E552E7CFD9FF1200D9CFE6FFE1CFD9FF06
:102EE000020EE126FE0EDB5020E1B3C0E9FFB4C0C4
:102EF000EAFFEE52080EEF6EB3C0E9FFB4C0EAFF7E
:102F0000020EE926000EEA22200EEE6E040EED6E91
:102F1000B3C0E9FFB4C0EAFF8C0EEF6EB9C0E9FFA1
:102F2000BAC0EAFF840EEF6E3DD0FD0EDB50E82400
:102F30000D6EFE0EDB50040DF3500D24040DF3CF87
:102F40000BF0F4CF0CF0000E0B26040E0C220BC07D
:102F5000DEFF0CC0DDFF840E0B6EDECFE9FFDDCFA0
:102F6000EAFF0B50EF12FD0EDB50E8240D6EFE0E53
:102F7000DB50040DF3500D24010F040DF3CF0BF0C3
:102F8000F4CF0CF0000E0B26040E0C220BC0DEFF5B
:102F90000CC0DDFF840E0B6EDECFE9FFDDCFEAFF54
:102FA0000B50EF12020EE15C02E2E16AE552E16EC3
:102FB000E552E7CFD9FF1200D9CFE6FFE1CFD9FF25
:102FC000020EE126FD0EDB500FE0FE0EEA6ADB3456
:102FD000FE0BEA36E96EB90EE926000EEA22EECFC4
:102FE000DEFFEDCFDDFF0ED0FE0EEA6ADB34FE0B16
:102FF000EA36E96EB50EE926000EEA22EECFDEFFD4
:10300000EDCFDDFFD9CFE9FFDACFEAFFEE50ED10CB
:1030100003E1F36AF46A49D0DECFE9FFDDCFEAFFCE
:10302000020EE926000EEA22FB0EDBCFEEFFFC0EBD
:10303000DBCFEDFFDECFE9FFDDCFEAFFEE52FA0E88
:10304000DBCFEFFF400E0B6EDECFE9FFDDCFEAFFF7
:103050000B50EF16880E0B6EDECFE9FFDDCFEAFFD7
:103060000B50EF12FD0EDB500CE0FE0EEA6ADB3473
:10307000FE0BEA36E96EB90EE926000EEA22EF747D
:103080000BD0FE0EEA6ADB34FE0BEA36E96EB50EB3
:10309000E926000EEA22EF74DECF0BF0DDCF0CF054
:1030A0000BC0F3FF0CC0F4FF00D0020EE15C02E2A3
:1030B000E16AE552E16EE552E7CFD9FF1200D9CFC0
:1030C000E6FFE1CFD9FF6DA84ED0FE0EEA6ADB34F1
:1030D000FE0BEA36E96EB90EE926000EEA22EE5042
:1030E000EFCFEAFFE96E400EEE16EE6AEE6AEE6A88
:1030F000FE0EEA6ADB34FE0BEA36E96EB90EE9260B
:10310000000EEA22EE50EFCFEAFFE96EEE7CFE0EF3
:10311000EA6ADB34FE0BEA36E96EB90EE926000EE8
:10312000EA22EF74400E0B6EFE0EEA6ADB34FE0BF1
:10313000EA36E96EB90EE926000EEA22EE50EFCF2C
:10314000EAFFE96E0B50EF16FE0EEA6ADB34FE0B67
:10315000EA36E96EB90EE926000EEA22EE50EFCF0C
:0E316000EAFFE96EEF7CE552E7CFD9FF1200DF
:02316E00DACFB6
:10317000E4FFE2CFDAFFE652E552E5CFDAFF1100D5
:10318000D8CFE4FFE0CFE4FFE46EDACFE4FFE2CF94
:10319000DAFFE652E552E5CFDAFFE550E5CFE0FF92
:1031A000E5CFD8FF100005D888EC10F017D8FCD771
:1031B00012000F0EC11202D81CEF10F09268936833
:1031C000F80E946E806A816A826A896A8A6A8B6A5A
:1031D0000001DC6BDD6BDE6BDF6B1200200E00018B
:1031E000E76EAE19E8AE02D0E73402D0E750AE5D2C
:1031F00003E36D50020B01E001D06BD81200D9CF70
:10320000E6FFE1CFD9FF030EE126010EDB6A020ED5
:10321000DB6AF29EDF6ADFCF0BF0080EE76E0B1859
:10322000E8AE02D0E73402D0E7500B5C2FE20A0E82
:10323000E66EF4EC1DF0E5529392FE0EDB50010BAE
:10324000E8B0948EE8A0949EFE0EDB407F0BE76E04
:10325000FE0EE7CFDBFF0A0EE66EF4EC1DF0E55242
:10326000010EDB407F0BE76E010EE7CFDBFFDBCF0C
:10327000E6FF8150010B800DF350E552E710E76E39
:10328000010EE7CFDBFF9382DF2AC5D781A611D0DD
:10329000020EDB2ADBCF0BF0640EE76E0B18E8AEF4
:1032A00002D00B3403D0E750D8800B5401E201D098
:1032B000EDD7F28E010EDB500B6E030EE15C03E2E4
:1032C00000D0E16AE552E16E0B50E552E7CFD9FF3D
:1032D0001200D9CFE6FFE1CFD9FF040EE126DF6A65
:1032E0009394DFCF0BF000016051E76E0B18E8AE4E
:1032F00002D0E73402D0E7500B5C2DE2DFCFE9FFCC
:10330000EA6AE9BEEA68610EE926000EEA22EF5099
:10331000E66E75DFE552E66EDFCFE9FFEA6AE9BEE9
:10332000EA68810EE926000EEA22E552E750EF6EC8
:103330000F0E00018215E824030F606F020EDF5CA0
:1033400008E15A0E835D05E09384050E606F6FD22D
:1033500001D0DF2AC6D793848251410A01E005D00B
:1033600084C0E1F085C0E2F000D00501006B016B84
:10337000036B046B056B066B076B0001E151200BBF
:1033800001E0010E040DF3CF0CF0E151800B01E0E0
:10339000010EE8240B6EE251100B01E0010E0B242C
:1033A0000C24E76E020EE7CFDBFFDB500EE0020ECF
:1033B000DBCF0BF0060EE76E0B18E8AE02D00B3435
:1033C00003D0E750D8800B5401E231D2E251020B16
:1033D00001E0010E080DF3CF0DF0E251080B01E002
:1033E000010E040DF3CF0CF0E251010BE8240B6E3B
:1033F000E251040B01E0010E0B240C240D24E76EB6
:10340000030EE7CFDBFFDB5001E111D2030EDBCF70
:103410000BF0090EE76E0B18E8AE02D00B3403D0A8
:10342000E750D8800B5413E2030EDBCF0CF00C0EE8
:10343000E76E0C18E8AE02D0E73402D0E7500C5C1F
:1034400006E2090EF36E030EF3CFDBFF12D0030E7C
:10345000DBCF0BF00C0EE76E0B18E8AE02D0E734B2
:1034600002D0E7500B5C05E30A0EF36E030EF3CFB8
:10347000DBFF0001AB5101E091D0AA054CE1010E48
:10348000E76EAD19E8AE02D0AD3503D0E750D88075
:10349000AD5541E3020EDBCF0BF0A951E76E0B18DF
:1034A000E8AE02D00B3403D0E750D8800B540BE2C7
:1034B000A90502E1040EAC6F0501510E026F000177
:1034C000A92B140EAB6FA90512E1010EE76EAC1922
:1034D000E8AE02D0AC3503D0E750D880AC5507E257
:1034E0000501520E026F0001AC07140EAB6F020E05
:1034F000DBCF0BF0A951E76E0B18E8AE02D0E73432
:1035000002D0E7500B5C07E20501520E026F00018A
:10351000A907140EAB6F030EDBCF0BF0AA51E76EB9
:103520000B18E8AE02D00B3403D0E750D8800B5410
:103530000DE2AA0502E1040EAD6F05014F0E026F08
:103540000001AA2B010EA96F140EAB6FAA0512E1A0
:10355000010EE76EAD19E8AE02D0AD3503D0E750ED
:10356000D880AD5507E20501500E026F0001AD078E
:10357000140EAB6F030EDBCF0BF0AA51E76E0B18E6
:10358000E8AE02D0E73402D0E7500B5C07E2050159
:10359000500E026F0001AA07140EAB6F0A0EAB5D4E
:1035A00002E10501026B0001AB51000801E2AB072B
:1035B0000001E2BF13D0640E0001E76EA219E8AE6D
:1035C00002D0E73402D0E750A25D01E2A22B0F0E39
:1035D000A25D04E1A56B010EA66FA46B0001E2AF32
:1035E0001BD0000E0001E76EA219E8AE02D0A23592
:1035F00003D0E750D880A2550DE20F0EE76EA21956
:10360000E8AE02D0E73402D0E750A25D03E2010E3B
:10361000A56FA46BA26BA66B0001A50517E1640E54
:10362000E76EA419E8AE02D0E73402D0E750A45DFB
:1036300001E2A42B050EE76EA419E8AE02D0A43572
:1036400003D0E750D880A45501E2A56B0001E1B199
:1036500013D0640E0001E76EA119E8AE02D0E73482
:1036600002D0E750A15D01E2A12B0F0EA15D04E1A4
:10367000A76B010EA86FA36B0001E1A11BD0000E88
:103680000001E76EA119E8AE02D0A13503D0E750E2
:10369000D880A1550DE20F0EE76EA119E8AE02D059
:1036A000E73402D0E750A15D03E2010EA76FA36BE0
:1036B000A16BA86B0001A70517E1640EE76EA319C3
:1036C000E8AE02D0E73402D0E750A35D01E2A32BBD
:1036D000050EE76EA319E8AE02D0A33503D0E7507C
:1036E000D880A35501E2A76B0001E1B703D0050123
:1036F000280E036F0001A70503E105012C0E036FDF
:103700000001A50503E10501500E036F0001E2BDB4
:1037100003D00501510E036F0001E2BB03D0050188
:103720004F0E036F0001A60503E10501520E036F62
:103730000001A80503E10501290E036F0A0EE66EDC
:10374000D6EC1DF0E5520001DC51DD1102E1000E66
:1037500008D0DCC0E9FFDDC0EAFFEF50800B01E0DC
:10376000010E000963E1010EDB6ADF6ADFCF0BF0B7
:103770000C6A0BBE0C68080E0B5C000E0C581CE2A9
:10378000DFCFE9FFEA6AE9BEEA68080EE926050E1E
:10379000EA22EFCF0BF0DFCFE9FFEA6AE9BEEA6881
:1037A000000EE926050EEA22EF500B5C03E0DE5224
:1037B000010EDD6EDF2ADAD7010EDB0413E1080EFD
:1037C000E66E000EE66E050EE66E010EE66EE66E25
:1037D000DCEC17F00B6E050EE15E0B50F3CFDCF066
:1037E000F4CFDDF0DF6ADFCF0BF00C6A0BBE0C68A4
:1037F000080E0B5C000E0C5819E2DFCFE9FFEA6AF5
:10380000E9BEEA68000EE926050EEA22EF50E66EF0
:10381000DFCFE9FFEA6AE9BEEA68080EE926050E8D
:10382000EA22E552E750EF6EDF2ADDD700D0040E22
:10383000E15C02E2E16AE552E16EE552E7CFD9FFD1
:1038400012001200120012001200FEEF1CF0120013
:103850001E0EE66E010EE66E36EC17F0E552E552EE
:1038600012006D840001080EE76F070EE86FE7078E
:10387000000EE85BE751E811FAE16D941200D9CF30
:10388000E6FFE1CFD9FFFD0EDBCF06F0FE0EDBCF6A
:1038900007F0720E061801E1075033E0E8680618D9
:1038A00002E17F0E07182BE0740E061801E10750A5
:1038B00024E0750E061801E107501DE0730E06188E
:1038C00001E1075016E0030E061801E107500FE072
:1038D000020E061801E1075008E0010E061801E18A
:1038E000075001E010D0B4DF0FD0B1DF0DD0ADDF55
:1038F0000BD0A9DF09D0A5DF07D0A4DF05D0A4DF56
:1039000003D0000001D000D0010E00D0E552E7CF77
:04391000D9FF1200C9
:0C3914001201000200000008D804550059
:1039200001000102000109022900010100C0320961
:103930000400000203010100092111010001223FDE
:1039400000070581030800010705010308000104C1
:1039500003090434034D006900630072006F0063C3
:103960000068006900700020005400650063006872
:10397000006E006F006C006F006700790020004946
:10398000006E0063002E002E034B0065007900627C
:10399000006F006100720064002000440065006D4B
:1039A000006F0000000000000000000000000000A8
:1039B000000000000005010906A101050719E02922
:1039C000E7150025017501950881029501750881AB
:1039D00003950575010508190129059102950175E1
:1039E000039103950675081500256505071900293B
:0C39F000658100C026394F3953398739F2
:0439FC000401205151
:103A00001F0B010801E068D0245101E065D0060ECB
:103A1000215D25E12351230A21E0010A11E0030A77
:103A200001E01DD00001AF050AE10001380EBF6FB3
:103A3000390EC06F090EC26FC36BC00EC16F0FD0BD
:103A40000001AF050AE10001B50EBF6F390EC06F6E
:103A50003F0EC26FC36BC00EC16F01D000D0040116
:103A60002051600BE842E842E842E842E84201089F
:103A700001E032D021510B0A29E0080A1CE0090AB2
:103A800014E0080A07E00B0A04E0080A01E024D069
:103A900023D022D00001F30EBF6F000EC06F010EC5
:103AA000C26FC36BC10EC16F17D00001800EC16F12
:103AB00023C4F3F011D00001F40EBF6F000EC06FED
:103AC000010EC26FC36B810EC16F06D00001800E64
:0A3AD000C16F22C4F4F000D0120010
:063ADA002A0EF66E200E1C
:103AE000F76E000EF86E00010900F550EE6F090048
:103AF000F550EF6F03E1EE6701D03DD00900F550BE
:103B0000E96F0900F550EA6F0900F550EB6F090005
:103B10000900F550E96E0900F550EA6E0900090048
:103B20000900F550EC6F0900F550ED6F0900090030
:103B3000F6CFF0F0F7CFF1F0F8CFF2F0E9C0F6FFF2
:103B4000EAC0F7FFEBC0F8FF0001EC5302E1ED53D0
:103B500007E00900F550EE6EEC07F8E2ED07F9D743
:103B6000F0C0F6FFF1C0F7FFF2C0F8FF0001EE076A
:083B7000000EEF5BBFD712004D
:083B7800FE0EE3CFE9FFFF0E92
:103B8000E3CFEAFFE9CFF3FFEACFF4FFFB0EE35008
:103B900003E1FC0EE35009E0FB0EE30602E2FC0E3B
:0C3BA000E306FD0EE350EE6EF1D71200BC
:043BAC00FF0EE350D5
:103BB0000E6E480E01D04C0EE76EE72EFED7E76A78
:0C3BC000E72EFED70E2EF7D700001200F3
:043BCC0013EE00F004
:103BD00023EE00F0F86A0A9C6DEC1DF006EC1EF076
:083BE000D3EC18F0FBD7120032
:083BE800FF0EE350E84E12004D
:0E3BF000000000D000D000D0E82EFAD712005E
:023BFE0000EED7
:0C3C000000F00F0EEE6AEA62FDD7120021
:023C0C001200A4
:023C0E000501AE
:103C10004200000000000000000000000000000062
:103C20000000000000000000000000000000000094
:103C30000000000000000000000000000000000084
:103C40000000000000000000000000000000000074
:0C3C500000000000000000010100000066
:020000040030CA
:0100000024DB
:010001000EF0
:010002003FBE
:010003001EDE
:010005008179
:010006008178
:010008000FE8
:01000900C036
:01000A000FE6
:01000B00E014
:01000C000FE4
:01000D0040B2
:00000001FF
